:02000000422894
:080008008C0003088D008E0B33
:100010003C283D308E00910A11080A3C031D3C2803
:1000200000309100920A1208063C031D3C28003063
:100030009200930A13080A3C031D3C2800309300E9
:10004000940A1408063C031D3C2800309400950ACD
:100050001508043C031D2D28352815080A3C031DEE
:100060003C2800309500960A3C281608023C031DE7
:100070003C280030950096000D0883008C0E0C0E75
:100080000B11090083168530810080308600F03026
:100090008500831286013D308E008101910192011D
:1000A0009301940195019601A0308B00861F752065
:1000B000051E8C205C2056281308AC2086000514F1
:1000C0009C2005101408AC20860085149C20851007
:1000D0001508AC20860005159C2005111608AC20DB
:1000E000860085159C2085110800950A1508043C9A
:1000F000031D7B28832815080A3C031D8A2800302D
:100100009500960A8A281608023C031D8A280030AA
:1001100095009600A4200800930A13080A3C031DCA
:100120009A2800309300940A1408063C031D9A286C
:1001300000309400A42008008F01053090008F0B40
:100140009F28900B9F2808008F010F3090008F0B85
:10015000A728900BA728080082073F3406345B3499
:0E0160004F3466346D347D3407347F34673499
:02400E00F13F80
:00000001FF
